:020000040000FA
:04000400AFEF01F069
:0600080000010AD91100FD
:10001800D8CF04F0E0CF05F0066EE9CF07F0EACFBD
:1000280008F000019DA279D09EA277D09E92822BE3
:10003800310E8261826B0B6A0C6A0D6A02EE41F026
:10004800D8900D34E926EF38E8461F0B030B0A6EEB
:1000580002EE40F0D8900D34E926EFCF09F00A50AF
:100068000CE0010A03E0030A05E007D085A505D0E6
:10007800096A03D085B501D0096AD8900950826110
:1000880001D0D8800C320B320D2A0F0E0D64D6D752
:100098008A510C1A89510B1A0BA089900BB08980D0
:1000A8000BA289920BB289820BA489940BB4898420
:1000B8000BA689960BB689860BA88A980BB88A88EE
:1000C8000BAA8A9A0BBA8A8A0BAC8A9C0BBC8A8CBC
:1000D8000BAE8A9E0BBE8A8E0CA08B920CB08B82C4
:1000E8000CA28B940CB28B840CA48A940CB48A84D2
:1000F8000CA68A960CB68A860CA88B900CB88B80B6
:100108000CAA8B980CBA8B880CAC8B9A0CBC8B8A7B
:100118000CAE8B960CBE8B86857585AD73D09DA86D
:1001280028D09EA826D09D98A0B905D086AD03D02A
:10013800A0812C801ED081A01CD00A6AA0B90BD047
:100148003B0EAF6E960E096E81B003D0010E0A6E9B
:1001580002D0092EF9D70A660AD001EE40F09A516A
:10016800E926EFCFADFFA0899A2B910702D0A08195
:100178002C809DAA47D09EAA45D0346A0B6AABA2B0
:1001880003D0AB98AB8832D0ABA409D0AE50010EE7
:100198000B6E86AF2BD03B0EAF6E869F27D0AECFAF
:1001A80009F009BE946B01EE00F09451E92609C0EC
:1001B800EFFF86AF04D03B0EAF6E869F12D0A0A98A
:1001C80010D001EE40F09951E926EFCF0AF009501E
:1001D8000A1803E0010E0B6E04D0992B999B9167C6
:1001E8009D880B6603D02C82942B949BA0A90AD0DF
:1001F8000B5208E0A0999D98A0812C80630EAF6EE9
:10020800AD6A868F07C0E9FF08C0EAFF065005C03F
:10021800E0FF04C0D8FF100085AF09D0F2A807D0CE
:10022800F2A205D0F292CF68640ECE6ECD8085AD75
:1002380011D0F2A80FD0F2A20DD0F292F298868DCA
:10024800346A2CB007D0A0B905D00D0E9D6102D03C
:10025800020E9D2785AF48D09DA046D09EA044D0D1
:100268009E90CD90E9CF00F0EACF01F0FACF02F0EE
:10027800FBCF03F0F9503E44F92603D00CD014D03C
:1002880024D081A006D03F2A090E3F6425D03E2AFB
:1002980023D03F6A21D081B01FD0680E3D6E676BB6
:1002A800080E416E3E2A18D0D89081B0D8804036CA
:1002B800412E12D03DC0E9FFEA6A40C0EFFF672B2C
:1002C8003D2A080E416E3E2A07D081B002D03E0674
:1002D80003D03E6A3F6A2C8A02C0FAFF03C0FBFFC4
:1002E80000C0E9FF01C0EAFF12004CBE09D0D6CF1A
:1002F8000EF04F500E5C505E0EC04FF0D8A04C8EE2
:100308001200D6CF0EF04D500E5C4E5E0EC04DF072
:10031800D8B012007D0E4E26050E0F6E010E106E1F
:1003280000EE42F04C5010140DE1EF06EF3C03D004
:10033800EE50EF06ED50EF50EE50EF1002E1105086
:100348004C12ED50020EE926000EEA22D890103623
:100358000F2EE8D71200000103D000EC78F000015E
:100368000F01BDEC10F056EC11F04C684D6A4E6A66
:10037800C60ED56E2C6A01EC12F02C862C88D08E15
:10038800F28EF28C2D6A2E6A2F6A306A800E3C6ECD
:10039800366E376E386E396E3A6E3B6E346E316E2D
:1003A800326E336E356E85AF03D0316AF292F288C1
:1003B800326A336A356A376A0400D190BA8495DFA5
:1003C800A0DF2DBE02D0F8DA2D6E2EBE02D000DBE3
:1003D8002E6E2FBE02D08ADB2F6E30BE03D0AAEC61
:1003E80005F0306E31BE04D00101ADD8316E000188
:1003F80032BE02D0B2D9326E33BE02D016DA336EB4
:1004080034BE02D06ED9346E35BE02D0D2D9356E24
:1004180036BE02D066DA366E37BE02D07DDA376E67
:1004280038BE03D017EC08F0386E39BE03D0CDECD7
:1004380008F0396E3ABE03D004EC06F03A6E3BBEC3
:1004480003D0B5EC07F03B6E3CBEB9D7F1EC05F034
:100458003C6EB5D785B34FD0F29ECF0E806EFC0EA2
:10046800816E3F0E826E480E0E6E020E0F6E106A7F
:10047800100E106020D00EC016F00FC017F002EE5C
:1004880000F0D8901034E926EF50DAEC0DF00E2A7F
:10049800000E0F220EC016F00FC017F002EE01F08A
:1004A800D8901034E926EF50DAEC0DF00E2A000E41
:1004B8000F22102ADDD7602B000E612362230EC0A5
:1004C80016F00FC017F06051DAEC0DF00E2A000E8E
:1004D8000F220EC016F00FC017F06151DAEC0DF0C4
:1004E8000E2A000E0F220EC016F00FC017F0625130
:1004F800DAEC0DF085832B0EC26EC2B2FED7030E66
:10050800C4148E6FC3CF8DF00E0E8D5D010E8E5903
:1005180009E2899E640E136E08D8898E640E136EE4
:1005280004D8E9D7D190FF001200146A1350146060
:1005380009D0A192B10EB36EB180A1A2FED7B1903D
:10054800142AF4D71200F9503144F92600D02CAA05
:10055800010C20EE67F000EE73F01F0EDF14626FDF
:100568006229DECFEEFFE806000AFBE12C9A656BF4
:10057800010E636F6251636108D0EA6A730E6325E6
:10058800E96EEF50651B632BF5D7EA6A730E632596
:10059800E96E6551EF62A1D074C067F167499DD0DB
:1005A800C00E6715D8B499D0400AD8B496D0C00AFE
:1005B80003E0400A73E091D0000175BF34D03F0ECC
:1005C8007415040DF3CF67F1060E7515D890E83051
:1005D800010167130001751D0101686F700E68172E
:1005E80068390F0B686F1F0E000176150101646FE3
:1005F800643B6443F80E6417645168136751000143
:100608008F6306D0010168510001906301D065D065
:1006180067C18FF068C190F067C187F068C188F042
:10062800386A01015AD03F0E74150101676F6707D8
:10063800D8906737D8906737070E00017515D8909E
:10064800E830010167130001751D0101686F700E24
:10065800681768390F0B686F010E000175190101E1
:10066800646F010E6417643B6443F80E64176451A9
:100678006813675100018F6306D0010168510001BA
:10068800906301D02AD067C18FF068C190F067C12C
:1006980087F068C188F0386A01011FD03F0E000159
:1006A80074150101686F75C067F16751606304D004
:1006B8006851616301D00AD0000185AB0ED00F0EDE
:1006C800010167630AD0270E686307D0EC0E0001AA
:1006D8007615EC0A02E187EC0CF00101000C01012F
:1006E800800CF9503444F92602D007D032D0868DD8
:1006F800D6CF4FF0960E506E4C9E4CAE010CF29237
:10070800F2889D450E6EF9500E44F926960E1DD0BE
:100718008E0E1BD0860E19D07F0E17D0780E15D0EE
:10072800700E13D0690E11D0610E0FD05A0E0DD075
:10073800520E0BD04A0E09D0430E07D03C0E05D0FE
:10074800340E03D02D0E01D0000ED6CF4FF0506ED0
:100758004C9E4CAE020C869D800C0101F95032442F
:10076800F92600D000012CA2010C010100AF1ED017
:1007780000DA0E6E0E50000119E0FF0A05E10101D2
:10078800006B0001A09912D011EE00F004EE00F009
:100798009251E926E6CFEEFFE950D8B404EE00F016
:1007A8000E2EF8D7E9CF92F0A0992C802C92000158
:1007B800000C3550D8A4800C9251931935E004EE02
:1007C80000F09351E926EFAE2ED004EE00F0E926B2
:1007D800EF50B00A07E05D0A12E0020A1DE05B0A6A
:1007E80020E021D0AEEC09F00EC087F00FC088F0F1
:1007F80087518815FF0A17E08591386A14D04FECA5
:1008080009F00EC087F00FC088F087518815FF0ADD
:100818000AE08581386A07D00701F0EC0AF0000188
:1008280002D0C2EC0DF0932B000C0101F9503344B7
:10083800F92605D004D030D039D03FD04DD00001B2
:100848002CA4010C2C94010140390F0B00019D6F61
:100858000F0E010140150001916F010E996F9A6FFB
:1008680085AF15D0040E946F526A915152600DD025
:1008780001EE41F05250E926EFCF53F001EE00F0BF
:10088800E92653C0EFFF522AF0D72C8228D086BD24
:1008980002D0A0B703D0020C0001F9D7D6CF4FF091
:1008A80084C050F04C9E4CBE03D0030C0001FBD713
:1008B8009D882C902CB003D0040C0001FBD7A0A17C
:1008C8000DD0A09186BDC4D7D6CF4FF084C050F0CC
:1008D8004C9E4CBEBDD7050C0001FBD79D6B2C86EA
:1008E800000CF9503644F92600D02CA6010C2C96A1
:1008F80011EE20F0E6CF0EF021EE40F00EC0DEFF44
:100908000E060F6AE6CFDFFFDE500F1A0E2EFAD75B
:100918000F1CDF6E2C84800CF9503744F92601D067
:1009280006D09751956303D09851961944E02CA6A8
:10093800010C2C9621EE40F09551E96E050E962596
:10094800EA6EEFCF0EF00EC0DEFF952B000E962359
:10095800956705D0020E966302D0956B966B0E06CE
:100968000F6A9551E96E050E9625EA6EEFCFDFFF07
:10097800DE500F1A952B000E9623956705D0020EB0
:10098800966302D0956B966B0E2EEBD70F1CDF6E1D
:100998009551975D0E6E965198590F6E0FAE02D015
:1009A800020E0F260FBE05D0D00E0E5C010E0F589A
:1009B800D8A02C882C84000CF9502D44F92601D09D
:1009C80004D0010E426E436A4C904CA0010C000CFE
:1009D800F9502E44F92603D006D009D018D00A0EB3
:1009E800446E456A4C924CA2010C2B0EC26EC2B2E8
:1009F800020C030EC4148E6FC3CF8DF08E5105E127
:100A0800FB0E8D6102D026DD0001130EC26EC2B24C
:100A1800030C030EC4148C6FC3CF8BF0810E8B5D57
:100A2800010E8C591DE3800E8B5D020E8C5918E265
:100A380085BB29D0070109A303D00001858702D00F
:100A480000018597070109AF03D00001858902D00D
:100A58000001859907010983098F0001858B13D04F
:100A680085AB11D085A703D00701098302D0070100
:100A78000993000185A903D00701098F02D0070156
:100A8800099F0001859B3B6A396A020101EC0FF05E
:100A980020EC0FF0000186AB04D0642F02D0869BB7
:100AA800898E85AD22D081B008D0A0A70DD09B2B10
:100AB8000A0E9B6309D0A09707D09B6BA0B704D000
:100AC8009C6702D0010E9C6F9C530FE09C2B180E64
:100AD8009C650BD09C6BF29EF292F288AB889E9A32
:100AE8009D8A9D98AC8AF28EA087000CF9502F44FD
:100AF800F92601D004D0640E466E476A4C944CA483
:100B0800010C8F6B906B65530EE065070F0E651532
:100B18000AE1653B65070F0E651504E0050E636F76
:100B28003C6A658B653B665307E0662F05D0050E6A
:100B3800636F3C6A010E666F86A107D086BB05D03D
:100B4800050E636F010E666F3C6A000CF950304465
:100B5800F92601D005D0E80E486E030E496E4C9672
:100B68004CA6010C896B8A6B80A802D089698A69B6
:100B7800000C00AD14D000AB0FD0020E0001946140
:100B880001D0000C01C10FF0030E01010F6403D066
:100B9800100E0F640BD0FF0C060E0F6E07D000ABC3
:100BA80003D0040E0F6E02D0020E0F6E0001945196
:100BB8000F6212D0106A116A01EE00F01150E92696
:100BC800EF50101A112A0F50115CF6E3102801019A
:100BD80002E10F501200FF0C000C3C50D8A4800C0E
:100BE80063C064F0868B899E800C972B000E982337
:100BF800976705D0020E986302D0976B986B120026
:100C0800F9503A44F92602D0BCD02ED15194546AF6
:100C1800200E54602BD1080E5402F350300F556E3D
:100C2800070E566A562255C0D9FF56C0DAFFDFAE06
:100C38001BD1040ED924E16E000EDA20E26E519227
:100C4800E6CF0FF0E7CF10F0116AE7BC112ADFB842
:100C580002D0E7AE2DD0DFA802D085B104D0DFB82E
:100C68002CD085B12AD00FC015F010C016F087C05F
:100C780017F088C018F01150CFDA1AC00EF00EBE67
:100C88001CD00EB00DD003EE80F05450E926EF9A38
:100C98000EB0EF8A03EE80F0E926EF900EB0EF80F9
:100CA80003EE80F05450E926EF900EB0EF8005D0A7
:100CB80003EE80F05450E926EF80060ED924E16E49
:100CC800000EDA20E26EE6CF0FF0E7CF10F0116ADF
:100CD800E7BC112ADFB602D0E7AE28D0DFA602D0E3
:100CE80085B104D0DFB627D085B125D00FC015F067
:100CF80010C016F087C017F088C018F011508CDAB1
:100D08001AC00EF00EBE17D003EE80F05450E9263C
:100D1800EFA004D003EE80F0E926EF8A03EE80F01E
:100D28005450E926EF920EB0EF8205D003EE80F022
:100D38005450E926EF821290DFBC128051B406D0DD
:100D4800545096D85192D8B0518206D003EE80F014
:100D58005450E926EF98EF9603EE80F05450E926B8
:100D6800EFB6518412B0519451A27DD0D9CFE1FF92
:100D7800DACFE2FFE4BE05D003EE80F0E926EFB853
:100D880072D02CA8010C55C0D9FF56C0DAFFD9CFB4
:100D9800E1FFDACFE2FF070EE4140FE0010A11E0E9
:100DA800030A13E0010A15E0070A17E0010A19E02F
:100DB800030A1CE0010A1FE022D0010E0E6E0F6A22
:100DC8001ED0050E0E6E0F6A1AD00A0E0E6E0F6A2E
:100DD80016D0320E0E6E0F6A12D0640E0E6E0F6AA7
:100DE8000ED0F40E0E6E010E0F6E09D0E80E0E6EC8
:100DF800030E0F6E04D0880E0E6E130E0F6EE738BA
:100E0800E8461F0B0F0B106E0E501002F3CF11F0B7
:100E1800F4CF12F0136A0F501002F3501226F45058
:100E2800132210AE04D00E50125E0F50135A0FAE9C
:100E380002D01050135E11501210131012E003EE7E
:100E480000F0030E5402F350E92611C0EEFF12C061
:100E5800EEFF13C0EEFF03EE80F05450E926EF8852
:100E680002D05450AFD8020C542AD2D6356A800C1E
:100E7800136E1590080E1302F350300FE16E070E33
:100E8800E26AE22203EE80F01350E926D890E730B8
:100E980006E3EFB002D0EFA206D0158004D0EFA091
:100EA80002D0EFB21580D890E730030B146E1450BF
:100EB80007E0010A1AE0030A2DE0010A38E04FD0E2
:100EC80015A010D0EFB403D015B003D006D015B0DC
:100ED80004D0EF86EF84D8801200EFB640D0EF86BA
:100EE800D8801200EF96EF943AD015B010D0EFB436
:100EF80003D015B003D006D015B004D0EF86EF9418
:100F0800D8801200EFB62BD0EF86D8801200EF966B
:100F1800EF8425D0EFB403D015B003D020D015B09E
:100F28001ED015A0EF9415B0EF84D880120015A03C
:100F380014D0EFBA02D0D8901200EFB403D015B095
:100F480003D006D015B004D0EF86EF84D880120005
:100F5800EFB605D0EF86D8801200EF96EF94D890C0
:100F68001200F9503B44F92602D006D024D0576A23
:100F7800200E576026D0010C03EE80F05750E9266A
:100F8800EFA81DD003EE00F0030E5702F350E92638
:100F9800EE06000EEE5AEF5A03EE00F0030E57026B
:100FA800F350E926EE50EE10EF1009E103EE80F061
:100FB8005750E926EF982CA8020C575003D8572A07
:100FC800D7D7800C146E080E1402F350300FE16E60
:100FD800070EE26AE222E7AA0FD0020EE126000E0F
:100FE800E222E6CF15F0166AE7CF16F015C017F023
:100FF80016C018F0DBD916D0020EE126000EE22248
:10100800E6CF15F0166A0F0EE714166E1688E7CFAE
:1010180017F017C025F0298015C026F016C027F054
:10102800000E50D21200F9503844F92601D007D0EA
:10103800800E356E586A200E5860A9D0010C080E33
:101048005802F350300FE16E080EE26AE222100EE9
:101058005824D96E070EDA6ADA22E6CF12F0136A3C
:10106800E7CF13F01490DFBE1480DF140F6E85B144
:1010780002D014A03FD012C015F013C016F087C0DC
:1010880017F088C018F0000EC7D81AC00EF00E2C42
:101098007CD0070E13161068116E12C015F013C01D
:1010A80016F010C017F011C018F098D8020E0F6291
:1010B8000CD003EE60F05850E9263C0EEF6E58C095
:1010C80015F0090E0AEC0EF062D0030E0F620CD078
:1010D80003EE60F05850E926140EEF6E58C015F074
:1010E800090E0AEC0EF053D058C015F0000E0AECA9
:1010F8000EF04DD085B149D014B047D0070E131467
:10110800166E1250156E87C017F088C018F0000EC2
:1011180083D81AC00EF00E6602D013A604D00E2C87
:1011280034D013A632D0F00E1316126A106A116E5C
:1011380012C015F013C016F010C017F011C018F047
:101148004DD8020E0F620CD003EE60F05850E9261D
:101158003C0EEF6E58C015F0090E0AEC0EF017D0D1
:10116800030E0F620CD003EE60F05850E926140EFF
:10117800EF6E58C015F0090E0AEC0EF008D058C0F2
:1011880015F0000E0AEC0EF002D0582A54D73A6A2D
:10119800800CF9503944F92601D005D0596A200E3F
:1011A80059601BD0010C03EE60F05950E926EF504E
:1011B80012E003EE60F05950E926EF0603EE60F006
:1011C800E926EF5008E15950B6EC0EF059C015F079
:1011D800080E0AEC0EF0592AE2D7800C28EE30F0FF
:1011E800196A200E196017D0DECF1AF0DDCF1BF078
:1011F80018501B1617501A161A50156206D01B5095
:10120800166203D01950B6EC0EF0080ED926000E5F
:10121800DA22192AE6D71200196E1A6885B102D0A7
:1012280085AF1AD01638E8461F0B1F0B1D6E1838ED
:10123800E8461F0B1F0B1E6E070E161618161550C4
:10124800176227D01650186224D01A6A1D501E62E1
:1012580020D0010E1A6E1DD01638030B1D6E1838DB
:10126800E840E8423F0B030B1E6E1D501E6211D072
:101278000F0E161618141C6E17501B6E15501B6295
:1012880008D016501C6205D01A6A18B81A2A1950C4
:101298001A1A1A501200932B04EE00F09351E92603
:1012A800EF500B0A03E00E680F68FF0C932B04EE57
:1012B80000F09351E926EF507F0A03E00E680F68AB
:1012C800FF0C932B04EE00F09351E926EF38070B3F
:1012D800030A03E00E680F68FF0C932B04EE00F07E
:1012E8009351E926070EEF14010A03E00E680F6810
:1012F800FF0C932B04EE00F09351E926EFCF0EF08C
:101308000EAC03D00E680F68FF0CD8900E36D8903C
:101318000E36932B04EE00F09351E926EFCF0FF031
:10132800700E0F1AD8900F32030E0F140E120F3AC8
:101338000F461F0E0F16932B04EE00F09351E9266B
:10134800EFCF10F0103A1042F80E101610500F128E
:101358000E50120004EE00F09351E926EFCF10F082
:10136800932B04EE00F09351E926D890EF340E6EDB
:10137800932B04EE00F09351E9263F0EEF140F6E05
:101388001190EFBC1180030E10140EE111A003D0D0
:101398000E680F68FF0CD8900F320E320FB603D0CC
:1013A8000E680F68FF0C0F960E5012009751E96EE9
:1013B800050E9825EA6E0B0EEF6EF9EC05F09751C5
:1013C800E96E050E9825EA6EED0EEF6EF9EC05F064
:1013D8009751E96E050E9825EA6E0B0EEF6EF9EC43
:1013E80005F09751E96E050E9825EA6E7F0EEF6EAF
:1013F800F9EC05F09751E96E050E9825EA6E310E65
:10140800EF6EF9EC05F01838E8441F0B196E183A1E
:101418001842F80E1816030E17141812D89018361A
:10142800700E181A1880189ED8901732D890173254
:101438009751E96E050E9825EA6E010EEF6EF9ECEC
:1014480005F09751E96E050E9825EA6E17C0EFFF73
:10145800F9EC05F09751E96E050E9825EA6E18C06B
:10146800EFFFF9EC05F09751E96E050E9825EA6E45
:1014780019C0EFFFF9EC05F09751E96E050E9825B4
:10148800EA6EEF6AF9EC05F09751E96E050E9825BA
:10149800EA6EEF6AF9EC05F09551975D196E965171
:1014A80098591A6E1AAE02D0020E1A261ABE06D023
:1014B800E10E195C010E1A58D8B02C98050E636F0E
:1014C8003C6A1200286E2538030B2A6E2B9027BE23
:1014D8002B801F0E271629B01DD02A5005E0010ABF
:1014E80006E0030A0EE015D02786279A35D02BA0F0
:1014F80002D028B01200279A278627A82DD0279631
:101508002BD02734273226322798D8B02788278A25
:1015180023D012002A5005E0010A09E0030A10E06E
:101528001AD02786100E25BC271A279A15D0279A75
:10153800100E25BC271A278627A80ED027960CD070
:101548002734273226322798D8B02788278A080ECA
:1015580025BC271A01D01200D89026362736D890F5
:1015680026329751E96E050E9825EA6E040EEF6E45
:10157800F9EC05F09751E96E050E9825EA6EB00E64
:101588002A10EF6EF9EC05F09751E96E050E9825D3
:10159800EA6E26C0EFFFF9EC05F09751E96E050EEB
:1015A8009825EA6E27C0EFFFF9EC05F09551975D95
:1015B8002A6E965198592B6E2BAE02D0020E2B260E
:1015C8002BBE06D0E10E2A5C010E2B58D8B02C9801
:1015D800050E636F3C6A120009A312000001932BE9
:1015E800932B04EE00F09351E9267C0EEF6268D04D
:1015F800932B04EE00F09351E926EFCF10F0932BD4
:10160800932B04EE00F09351E926EFCF0FF0932BC4
:1016180004EE00F09351E926D890EF340E6E0F34A3
:101628000F320E320E500101606304D00F50616317
:1016380001D00BD0000185AB07D00F0E0E6204D08D
:10164800270E0F6201D001D012000001932B932BBB
:10165800FC0E1014200A0BE0080A09E0040A14E042
:101668004C0A1FE0080A1DE00C0A23E029D00701F4
:1016780009AF07D010C011F00EC012F00FC013F060
:1016880020D8010E42DA1CD010C011F00EC012F0A2
:101698000FC013F016D809AF02D0010E36DA0001D8
:1016A8000FD031D9070109AF02D0400E2EDA000160
:1016B80007D029D9070109AF02D0400E26DA000168
:1016C800120011EE20F00E0EE66EE70EE66E0E0E1C
:1016D800E66E7C0EE66E11C0E6FFE66AD89012361A
:1016E8001336D890123213C0E6FF12C0E6FFE66A3E
:1016F8001A6A04EE00F000019351E926EFCF18F0C2
:1017080018C017F017380F0B176E932B04EE00F064
:101718009351E926EFCF19F019C016F0169E18B0AC
:10172800168E1B90165017100AE1060E166E176AD1
:10173800E96E070E1724EA6EEFCF1AF01B801750D8
:1017480003E1050E166412D0175010E1090E166059
:101758000DD0060E165E000E175A1650E96E070ECB
:101768001724EA6EEFCF1AF01B80B9D0100E16625C
:1017780002D0175205E0110E16620FD017660DD071
:101788000C0E165E000E175A1650E96E070E172437
:10179800EA6EEFCF1AF01B80A2D01B0E166202D0A1
:1017A800175205E01C0E16620FD017660DD0150EE5
:1017B800165E000E175A1650E96E070E1724EA6EC9
:1017C800EFCF1AF01B808BD0175003E11F0E166461
:1017D80013D0175011E1400E16600ED0200E165E81
:1017E800000E175A100E1624E96E070E1720EA6E1F
:1017F800EFCF1AF01B8073D06F0E16620FD01766EA
:101808000DD0660E165E000E175A1650E96E070EBA
:101818001724EA6EEFCF1AF01B8061D0175003E14E
:101828006F0E166413D0175011E1730E16600ED0A8
:10183800500E165E000E175A480E1624E96E090E51
:101848001720EA6EEFCF1AF01B8049D0730E16628C
:101858000ED017660CD0166A176A300E1624E96E79
:10186800090E1720EA6EEFCF1AF01B8038D01750F8
:1018780002E116AE13D0175011E1900E16600ED08B
:10188800800E165E000E175A380E1624E96E090EE1
:101898001720EA6EEFCF1AF01B8021D017520EE006
:1018A800020E17600BD01706300E1624E96E070ECD
:1018B8001720EA6EEFCF1AF01B8011D0010E1764C3
:1018C8000ED0030E17600BD0020E175E300E1624D2
:1018D800E96E080E1720EA6EEFCF1AF01B801892F7
:1018E8001ABE188218C0E6FF19C0E6FF7F0E1A1448
:1018F800E66EE66AE66A1BA003D0050E636F3C6AD3
:10190800A08B07011200159085AF0CD00C0E761530
:101918000C0AD8A41200030E7615146E77C013F0C3
:1019280078C011F085AD1DD004EE00F09351E92682
:10193800EFCF14F0932B04EE00F09351E926EFCF8C
:1019480013F0139E14B0138E932B04EE00F09351F2
:10195800E926EFCF11F0119E14B2118E14380F0B37
:10196800146E14502FE1200E13602CD0100E136249
:1019780002D0145205E0110E13620ED014660CD07A
:101988000C0E135E000E145A1350E96E070E142441
:10199800EA6E11C0EFFFACD01B0E136202D01452D6
:1019A80005E01C0E1362A4D01466A2D0150E135EB7
:1019B800000E145A1350E96E070E1424EA6E11C073
:1019C800EFFF96D0145003E11F0E136416D0145085
:1019D80014E1400E136011D0200E135E000E145A4D
:1019E800100E1324E96E070E1420EA6E11C0EFFFE3
:1019F800100E1326000E14227BD06F0E136214D023
:101A0800146612D0660E135E000E145A1350E96E57
:101A1800070E1424EA6E11C0EFFF859711B285876F
:101A2800859911BE858964D0730E136211D014662E
:101A38000FD0136A146A300E1324E96E090E1420AD
:101A4800EA6E11C0EFFF300E1326020E142250D09A
:101A5800145002E113AE16D0145014E1900E136026
:101A680011D0800E135E000E145A380E1324E96E3E
:101A7800090E1420EA6E11C0EFFF380E1326020E6D
:101A8800142236D0145211E0020E14600ED014063F
:101A9800300E1324E96E070E1420EA6E11C0EFFF12
:101AA800300E1326000E142223D0010E14641FD00A
:101AB800030E14601CD0020E145E1350126E1450E4
:101AC800176E030E166E17321232162EFCD71250EE
:101AD80049D9300E1324E96E080E1420EA6E11C09D
:101AE800EFFF300E1326010E1422158001D01200CC
:101AF80013C016F014C017F0115058D815B001ECE7
:101B080012F0050E636F3C6A1200116E00019751C6
:101B1800E96E050E9825EA6E040EEF6EF9EC05F0F5
:101B28009751E96E050E9825EA6EB40EEF6EF9EC42
:101B380005F09751E96E050E9825EA6E6F0EEF6E67
:101B4800F9EC05F09751E96E050E9825EA6E11C07B
:101B5800EFFFF9EC05F09551975D126E9651985983
:101B6800136E13AE02D0020E132613BE06D0E10E7A
:101B7800125C010E1358D8B02C981200932B04EE67
:101B880000F09351E9266F0EEF6204D0A0AB02D0AB
:101B9800A09B366A1200A6B2FED719C0A9FF1AC0C8
:101BA800AAFFA69EA69CA680A8501200186E16C072
:101BB80019F017C01AF0EFDF18181CE0A6B2FED70C
:101BC80018C0A8FF16C0A9FF17C0AAFFA69EA69C0A
:101BD800A684F29E550EA76EAA0EA76EA682F28E56
:101BE800A69416C019F017C01AF0D5DF181802E02D
:101BF800D8901200D880120014C0F6FF15C0F7FF65
:101C0800F86AA68EA69C0800F5501200166E209061
:101C1800080E1502F350300FE16E080EE26AE22258
:101C2800E6CF1CF0E5CF1DF015C017F0200E1760A9
:101C380095D01C50E6628CD01D50E76289D0100EFA
:101C48001724E96E070EEA6AEA22EF141B6E090EE2
:101C5800166204D0010E186EE65002D0040E186EFB
:101C6800E6500F0EE714196EE7B802D020A00AD08C
:101C780019B003D01B861B98208019A003D01B968F
:101C88001B882090080E166204D0030E186201D03B
:101C980028D0E738D890E830070B1A6E040E1A627D
:101CA80001D01FD0E00EE7141B101F6E380E192448
:101CB800E96E090EEA6AEA22EFCF1EF002EE00F0A2
:101CC800D8901934E9261EC0EEFF1FC0EEFF1BA4F2
:101CD80006D002EE70F01950E92630C9EFFF070E62
:101CE8001B16182EBDD71650090A36E0100E1724F9
:101CF800E96E070EEA6AEA22EF38D890E830030B5B
:101D0800010A11E0030A05E0010A0DE0030A06E0F2
:101D18000AD0030EE126000EE2221ED0030EE126B1
:101D2800000EE22219D0E4CF21F0226A0F0EE4144B
:101D3800226E2288E7CF23F023C025F0298021C016
:101D480026F022C027F0000E66EC0AF0E65004D018
:101D5800070EE126000EE222172A68D7050E636FE8
:101D68003C6A12001C6E080E1C02F350300FE16E24
:101D7800080EE26AE222E6CF20F0E7CF21F0040E57
:101D88001D6EE6500F0EE7141E6EE738D890E83047
:101D9800070B1F6E040E1F6201D007D002EE00F081
:101DA800D8901E34E926EE6AEF6A1D2EEAD7100E87
:101DB8001C24E96E070EEA6AEA22EF38D890E83068
:101DC800030B010A19E0030A04E0010A02E0030A0E
:101DD80013E0E4CF22F0236A0F0EE414236E238865
:101DE800E7CF24F024C025F0298022C026F023C0A4
:101DF80027F0000E66EF0AF01200809B80B5808BFA
:101E08005A2A320E5A6403D0010E5A6E8075809990
:101E180080B380895B2A4B0E5B6403D0010E5B6E36
:101E28008073809780B180875C2A640E5C6403D0DD
:101E3800010E5C6E807112000F6A100E0F6098D14F
:101E480002EE00F0D8900F34E926EECF13F0EECF73
:101E580014F01450166E156A1438D890E830070B31
:101E6800116E115011E0010A19E0030A35E0010A68
:101E780051E0070A6DE0010A73E0030AD8B48ED076
:101E8800010AD8B4A9D0C5D002EE20F0D8900F34FA
:101E9800E92613C0EEFF14C0EEFFBBD080A112D01C
:101EA80002EE20F0D8900F34E92613C0EEFF14C0DC
:101EB800EEFF80B7AED002EE70F00F50E92630C9C1
:101EC800EFFFA7D002EE20F0D8900F34E92615C016
:101ED800EEFF16C0EEFF9DD080A312D002EE20F0D8
:101EE800D8900F34E92613C0EEFF14C0EEFF80B976
:101EF80090D002EE70F00F50E92630C9EFFF89D07C
:101F080002EE20F0D8900F34E92615C0EEFF16C077
:101F1800EEFF7FD080A512D002EE20F0D8900F34CB
:101F2800E92613C0EEFF14C0EEFF80BB72D002EEAC
:101F380070F00F50E92630C9EFFF6BD002EE20F0A9
:101F4800D8900F34E92615C0EEFF16C0EEFF61D019
:101F580002EE20F0D8900F34E926EE6AEF6A59D0E5
:101F680080B112D002EE20F0D8900F34E92613C0C9
:101F7800EEFF14C0EEFF80A74CD002EE70F00F50B9
:101F8800E92630C9EFFF45D002EE20F0D8900F3493
:101F9800E92615C0EEFF16C0EEFF3BD080B312D085
:101FA80002EE20F0D8900F34E92613C0EEFF14C0DB
:101FB800EEFF80A92ED002EE70F00F50E92630C94E
:101FC800EFFF27D002EE20F0D8900F34E92615C095
:101FD800EEFF16C0EEFF1DD080B512D002EE20F045
:101FE800D8900F34E92613C0EEFF14C0EEFF80AB83
:101FF80010D002EE70F00F50E92630C9EFFF09D07B
:1020080002EE20F0D8900F34E92615C0EEFF16C076
:10201800EEFF02EE20F0D8900F34E926EECF17F04D
:10202800EECF18F002EE41F0D8900F34E926070EF3
:10203800EF14126E12521AE0040E126017D002EE5C
:1020480040F0D8900F34E9261750EF1804E0070E37
:102058001214106E15D002EE41F0D8900F34E92614
:1020680018C0EFFF070E1814106E0AD002EE41F0E8
:10207800D8900F34E92618C0EFFF070E1814106E19
:10208800105009E0010A11E0030A0FE0010A0DE00F
:10209800070A50E06BD002EE40F0D8900F34E926E2
:1020A80017C0EEFF18C0EEFF61D002EE40F0D890E6
:1020B8000F34E9261750EF6006D002EE40F0D890B2
:1020C8000F34E926EF2A02EE40F0D8900F34E926C3
:1020D800EF5017604BD002EE40F0D8900F34E9264D
:1020E800230EEF6407D002EE40F0D8900F34E926B3
:1020F800230EEF6E380E0F24E96E090EEA6AEA2203
:10210800EF503008E83AE8461F0B0E6E02EE60F01A
:102118000F50E926EF2A0E50EF5C28E302EE60F03C
:102128000F50E926EF6A02EE40F0D8900F34E92606
:10213800EF061CD002EE70F00F50E926EF500FE0CA
:1021480002EE40F0D8900F34E92617C0EEFF18C011
:10215800EEFF02EE70F00F50E926EF0607D002EE10
:1021680040F0D8900F34E926EE6AEF6A0F2A65D658
:102178001200F00ED36EC00E9B6E100E386F020E5A
:10218800396F3A6B110EC26EC16ABE0EC06E796AA3
:10219800786ACF0E806E300E926EFC0E816E030E42
:1021A800936E616A3F0E826EC00E946E2B0EC26EE5
:1021B8000001C2B2FED7030EC4148E6FC3CF8DF0D8
:1021C800220E8D5D010E8E590BE2899E640E136EF0
:1021D80099EC02F0898E640E136E99EC02F0E6D742
:1021E800AC9A3B0EAF6EAC98AB8EAB98B888AC94FB
:1021F800B896F26AF16AF06A9D6AA06A010E9F6E4B
:10220800A26AD59ED66A340ECD6E9E909D807E0EB3
:10221800BA6E1A0EBB6E9E929D82BA94300EB16E43
:10222800A68EA69CF66AF76AF86A0EEE00F0400ED3
:102238000E6E0900F552F5CFEEFF0E2EFAD70E6A94
:10224800010E116E0EEE00F00E50E926EFCF0FF0E2
:1022580002EC7BF0106E0F501062116A0E2A070E06
:102268000E64F0D7116612000E6A080E0E600CD0CC
:102278000E5002EC7BF00F6E0EEE00F00E50E926C9
:102288000FC0EFFF0E2AF1D7D1D8D8B01200899E1F
:10229800960E136E99EC02F0898E960E136E99ECD9
:1022A80002F0F2D7146AB50E156EA6DC126E196A22
:1022B8001A6A71DC121809E012C0A8FFA684550E2C
:1022C800A76EAA0EA76EA682A69407EE00F00E6A65
:1022D8000F6A0EC019F00FC01AF05DDCEE6E0E2A00
:1022E800000E0F22700E0E5C020E0F58F2E3106AF9
:1022F800116A0E6A0F6A0F502FE1100E0E602CD073
:10230800480E1024E96E090E1120EA6EEFCF13F083
:10231800D8900E34E96E0F34EA6E020EEA2613C026
:10232800EFFF102A000E1122480E1024E96E090E44
:102338001120EA6EEFCF13F0D8900E34E96E0F3407
:10234800EA6EE92A020EEA2213C0EFFF102A000EF5
:1023580011220E2A0F22CFD768C960F069C961F02F
:102368006AC962F03F0E070104150101616F05C7D4
:1023780060F1A68EA69CF66AF76A200EF86E0EEE3D
:1023880040F0080E146E0900F5CFEEFF142EFBD7AF
:1023980045CE48FE0001896B8A6B80A802D0896906
:1023A8008A69130EC26EC2B2FED7030EC4148C6FB4
:1023B800C3CF8BF086938691859F859D200E8B5D7C
:1023C800010E8C5902E2858D17D0220E8B5D010E0D
:1023D8008C5907E3800E8B5D010E8C5902E2858FC4
:1023E8000BD0820E8B5D010E8C5906E3800E8B5D3F
:1023F800020E8C59D8A08681120001016039F00BB9
:102408000001846F166A200E16600DD0080E1602A1
:10241800F350300FD96E080EDA6ADA221F0EDF1475
:102428008427162AF0D784C006F71200020E146E0D
:10243800A68EA69CA684A68EF66AF76AF86AA6886F
:10244800550EA76EAA0EA76EA682A6980A000EEED3
:1024580000F0400E136EEECFF5FF0F00132EFBD7E2
:10246800550EA76EAA0EA76EA682A694F66A0EEE61
:1024780000F01580400E136E0900F550EE1802E0CA
:10248800159002D0132EF8D715A002D0D8801200CC
:08249800142ED0D7D8901200D9
:10F000000001FFD729DA02EF00F01200186A17504A
:10F01000186009D09E90B10ECF6ECD809EA0FED715
:10F02000CD90182AF4D71200898E166A15501660F2
:10F030000AD0899E0A0E176EE9DF898E280E176E98
:10F04000E5DF162AF3D7C80E176EE0DFEDD7F29E84
:10F05000F29CF00ED36EC00E9B6E3B0EAF6EAC9862
:10F06000AB8EB888AB88100E386F020E396F3A6BD2
:10F07000110EC26EC16ABE0EC06E800E806E200E72
:10F08000926E816AF30E936E826AFC0E946E300E5D
:10F09000CD6E0FEE37F0ED6AEA50FDE1E950FBE18D
:10F0A000EF6A130EC26E000186930F01C2B2FDD744
:10F0B000030EC414166EC3CF15F0010E155C030EBB
:10F0C000165802E3000186830F0112000EEE59F07C
:10F0D0009351E926EFCF17F00EEE59F0E926EF6ACB
:10F0E000932B400E9361936B175012000E0EEA6E35
:10F0F00018501724E96EEFCF1CF0192C02D01B6AB0
:10F10000000C18C01DF01D2A1D501A6201D01D6A86
:10F110000E0EEA6E1D501724E96EEFCF1BF01B5048
:10F12000100A03E0FD0E1B6EFD0C1C6A0E0EEA6E4B
:10F1300018501724E96EEF501C1A182A18501A623A
:10F1400001D0186A1B041D6E1D521FE0190619BE5E
:10F1500002D0196602D01B6A000C0E0EEA6E18501F
:10F160001724E96EEFAE03D0FE0E1B6EFE0C0E0EE2
:10F17000EA6E18501724E96EEF501C1A182A18501E
:10F180001A6201D0186A1D06DFD71C3C02D01B5042
:10F1900012001B68FF0C9EAA14D0ABA203D0AB9840
:10F1A000AB880FD0ABA402D0AE500BD0899E0EEE30
:10F1B00059F09251E926AECFEFFF922B400E9261AB
:10F1C000926B9351925D156E15AE02D0400E1526CE
:10F1D000155224E00EEE59F09351E926E50EEF6248
:10F1E0001CD0590E176E93C018F015C019F0400EC0
:10F1F0001A6E7CDF1BC091F0915110E0FD0A05E012
:10F20000030A03E0010A03E004D060DF07D01668B8
:10F21000FF0C898E010E166E010C58DF166A000C69
:10F22000A6B2FED715C0A9FF16C0AAFFA69EA69C2F
:10F23000A680A8501200020E216EA69EA69CA6844F
:10F240001CC0A9FF1DC0AAFF0EEE49F01FC020F090
:10F25000EFCFA8FF550EA76EAA0EA76EA682A6B284
:10F26000FED7A680A850EF6209D0020E216EEE50A4
:10F27000A92AA950D8B4AA2A228002D0229002D06A
:10F28000202EE6D722A002D0D8801200212EE0D76F
:10F29000D8901200899E020E296EA68EA69CA68486
:10F2A000A68E24C0F6FF25C0F7FF26C0F8FFA6886B
:10F2B000550EA76EAA0EA76EA682A6980A000EEE9D
:10F2C00099F027C028F0EECFF5FF0F00282EFBD7CE
:10F2D000550EA76EAA0EA76EA682A69424C0F6FFAE
:10F2E0000EEE99F02A8027C028F00900F550EE189C
:10F2F00002E02A9002D0282EF8D72AA004D08687D0
:10F30000898ED8801200292ECAD7D8901200A68ED6
:10F31000A69C2650F86E2550F76EC00E2414F66E8B
:10F320000EEE99F0400E276E0900F5CFEEFF272E66
:10F33000FBD712003F0E1C14236E990E2324216E5E
:10F340002106490E226E236A1F50235C23501F188A
:10F35000D8B0800A36E6212AD90E216219D0990E3A
:10F36000216E87C024F088C025F0266A400E276EE3
:10F3700091DF0CE3400E8727000E882387C024F01E
:10F3800088C025F0266AC3DF869702D0D890120085
:10F390000E0EEA6E22C0E9FFEFCF20F01D501E10C6
:10F3A00003E1030E1C6406D00E0EEA6E21C0E9FFD5
:10F3B00020C0EFFF222A1C2A000E1D221E22232A13
:10F3C000C3D7D880120017501B6E16501A6EC00E8D
:10F3D0001514196E898E1B502CE1F00E1A6029D07D
:10F3E00086A70BD019C087F01AC088F087C024F018
:10F3F00088C025F0266A8BDF8697195087630ED068
:10F400001A5088630BD01B6609D015C01CF016C0BB
:10F410001DF017C01EF018C01FF08CD787C024F055
:10F4200088C025F0266A400E276E34DFD3E2D890DC
:10F430001200200E176002D0D8901200F00E176252
:10F4400009D015C01CF016C01DF017C01EF018C062
:10F450001FF0F1D6D880120014920F01F8DD0001E0
:10F4600086A312008687899E148095DEFF0A03E03A
:10F47000FE0A07E0BFD014A2BDD0040E156ED4DD85
:10F48000B9D0899E23DE22DE100AD8A4B3D01EDEB6
:10F490007F0AD8A4AFD01ADE7F0AD8A4ABD016DE7C
:10F4A0007F0AD8A4A7D012DE0E6E040E9325106E2C
:10F4B0003F0E106402D0400E105E0EEE59F0105058
:10F4C000E926F00EEF1408E0100A47E0300A55E094
:10F4D000600AD8B480D08ED0F9DD570A03E0010E5F
:10F4E000156EA2DDF3DD150A03E0010E156E9CDD3D
:10F4F000EDDD7F6F7F9F0EB47F8F020E9325106E20
:10F500003F0E106402D0400E105E0EEE59F0105007
:10F51000E926EFCF0FF00FA00FD00FB207D07F5129
:10F52000060A0AE0020E156E7FDD06D0060E7F6128
:10F5300003D0020E156E78DDC9DD7F6F7F9F0EB69A
:10F540007F8F0FA408D0156A166A6ADE7F6103D028
:10F55000030E156E69DD14824DD0B8DD136E139E57
:10F560000EB0138EB3DD126E129E0EB2128EAEDD91
:10F57000116E119E0EB4118E3DD01EEE49F0106A30
:10F58000040E106009D0A2DDE76E0E32D8A0E69E10
:10F59000D8B0E68E102AF4D799DD0F6E106A040EEB
:10F5A000106009D093DDE76E0F32D8A0E69ED8B088
:10F5B000E68E102AF4D711C015F012C016F013C051
:10F5C00017F0080E186EFFDE15E3080E1126000E68
:10F5D000122213220FD086B70CD087C024F088C027
:10F5E00025F0266A400E276E55DE03E2050E156EE5
:10F5F0001BDD149014B039D7898ECD6AAB6AAC6A22
:10F600009E6A1200136E180FF66EF60EF76AF72256
:10F61000F86A0800F550120002EF78F0AFEF01F041
:10B5000010571500270F00E0009F0000000000000A
:0200000400F00A
:1000000010571500270F00E0009F000000000000BF
:1000100000000000000000000000000000000000E0
:1000200000000000000000000000000000000000D0
:1000300000000000000000000000000000000000C0
:1000400000000000000000000000000000000000B0
:1000500000000000000000000000000000000000A0
:100060000000000000000000000000000000000090
:100070000000000000000000000000000000000080
:100080000000000000000000000000000000000070
:100090000000000000000000000000000000000060
:1000A0000000000000000000000000000000000050
:1000B0000000000000000000000000000000000040
:1000C0000000000000000000000000000000000030
:1000D0000000000000000000000000000000000020
:1000E0000000000000000000000000000000000010
:1000F0000000000000000000000000000000000000
:1001000000000000000000000000000000000000EF
:1001100000000000000000000000000000000000DF
:1001200000000000000000000000000000000000CF
:100130000800028282820030090001818181003042
:100140000808008080800030090803838383003022
:100150000A004282828200300B004181818100309E
:100160000A084080808000300B084383838300307E
:100170000C100686868600300D10058585850030BA
:100180000C180484848400300D180787878700309A
:100190000E104686868600300F1045858585003016
:1001A0000E184484848400300F18478787870030F6
:1001B00010200A8A8A8A0030112009898989003032
:1001C000102808888888003011280B8B8B8B003012
:1001D00012204A8A8A8A003013204989898900308E
:1001E000122848888888003013284B8B8B8B00306E
:1001F00014300E8E8E8E003015300D8D8D8D0030AA
:1002000014380C8C8C8C003015380F8F8F8F003089
:1002100016304E8E8E8E003017304D8D8D8D003005
:1002200016384C8C8C8C003017384F8F8F8F0030E5
:100230000A2E2E2E2E2E2E2E2F2F2F2F2F2F2F2FFA
:100240002F2F2F2F2F2F2F2F000000000000000036
:10025000000000000000000000000000000000009E
:10026000000000000000000000000000000000008E
:020000040000FA
:020000000000FE
:020000040030CA
:08000000FF280108FF8181FFC8
:00000001FF
